:1000000044EF21F0FFFFFFFF280E0101136F6E0E7A
:10001000146F750E156F6C0E166F6C0E176F290E20
:10002000186F196B216B226B1F6B206B01010EC1C6
:1000300000F00FC101F010C102F0010E0E27000EFA
:100040000F23102300C0F6FF01C0F7FF02C0F8FF26
:100050000900F5CF00F000C01CF10052D8B444EF05
:1000600011F01C51250A0BE00CC1E1FF0DC1E2FFAC
:100070001CC1E6FF0C4B0D2B214B222BD7D71D6B40
:100080001E6B1F6B206B010123D01F87010E0E27F3
:10009000000E0F2310235AD01F81010E0E27000ED1
:1000A0000F23102353D01F83010E0E27000E0F23A2
:1000B00010234CD02087010E0E27000E0F23102393
:1000C00045D01F85010E0E27000E0F2310233ED0B2
:1000D00001010EC1F6FF0FC1F7FF10C1F8FF0900C3
:1000E000F5CF2DF12D512D0AD0E00EC1F6FF0FC135
:1000F000F7FF10C1F8FF0900F5CF2DF12D51200AAF
:10010000CBE00EC1F6FF0FC1F7FF10C1F8FF0900E9
:10011000F5CF2DF12D512B0AC6E00EC1F6FF0FC110
:10012000F7FF10C1F8FF0900F5CF2DF12D51230A7B
:10013000C1E00EC1F6FF0FC1F7FF10C1F8FF0900C3
:10014000F5CF2DF12D51300ABCE001D09CD7010133
:100150001FB31F911FB71F950EC1F6FF0FC1F7FF09
:1001600010C1F8FF0900F5CF00F0000E016E00C0CD
:1001700000F1FCEC26F0005238E001011D6B1E6B13
:100180001DC100F01EC101F00A0E046E000E056EC6
:1001900091EC25F00EC1F6FF0FC1F7FF10C1F8FF7B
:1001A0000900F5CF2DF101012D5100241D6F000E26
:1001B00001201E6F300E1D5F000E1E5B010E0E270C
:1001C000000E0F2310230EC1F6FF0FC1F7FF10C161
:1001D000F8FF0900F5CF00F0000E016E00C000F13D
:1001E000FCEC26F00052CCE136D00EC1F6FF0FC178
:1001F000F7FF10C1F8FF0900F5CF2DF101012D51D6
:100200002A0A29E111C1E9FF12C1EAFFEECF00F08D
:10021000EECF01F000C0E9FF01C0EAFFEECF1DF113
:10022000EECF1EF111C1E9FF12C1EAFFEECF00F0DF
:10023000EECF01F0020E0026000E012211C1E1FFF7
:1002400012C1E2FF00C0E6FF01C0E6FF010E0E276B
:10025000000E0F23102301010EC1F6FF0FC1F7FF9F
:1002600010C1F8FF0900F5CF2DF12D512E0A74E1D0
:10027000010E0E27000E0F2310230EC1F6FF0FC133
:10028000F7FF10C1F8FF0900F5CF2DF12D512A0A13
:100290002AE111C1E9FF12C1EAFFEECF00F0EECF73
:1002A00001F000C0E9FF01C0EAFFEECF1AF1EECF86
:1002B0001BF111C1E9FF12C1EAFFEECF00F0EECF52
:1002C00001F0020E0026000E012211C1E1FF12C151
:1002D000E2FF00C0E6FF01C0E6FF010E0E27000EA0
:1002E0000F23102337D01A6B1B6B0EC1F6FF0FC103
:1002F000F7FF10C1F8FF0900F5CF00F0000E016E06
:1003000000C000F1FCEC26F0005224E01AC100F01D
:100310001BC101F00A0E046E000E056E91EC25F073
:100320000EC1F6FF0FC1F7FF10C1F8FF0900F5CFAE
:100330002DF101012D5100241A6F000E01201B6FB9
:10034000300E1A5F000E1B5B010E0E27000E0F23EE
:100350001023CBD7010104D001011A6B1B6B20893C
:1003600001010EC100F00FC101F010C102F0010E39
:100370000E27000E0F23102300C0F6FF01C0F7FF69
:1003800002C0F8FF0900F5CF1CF1EDD021C100F04B
:1003900022C101F012001F89E3D720851FD11F8BD6
:1003A00020811CD120831AD11F8D18D117D11F8B0A
:1003B0001F8F14D111C1E9FF12C1EAFFEECF00F087
:1003C000EECF01F000C0E9FF01C0EAFFEECF29F156
:1003D000EECF2AF111C1E9FF12C1EAFFEECF00F022
:1003E000EECF01F0020E0026000E012211C1E1FF46
:1003F00012C1E2FF00C0E6FF01C0E6FF000E2A19AD
:1004000002E1000E291904E1130E296F010E2A6F73
:1004100001012B6B2C6B2B512925E96E2C512A21C4
:10042000EA6EEECF00F0005203E02B4B2C2BF3D7FB
:100430001A511B110AE02C511B5D02E12B511A5D70
:1004400004E21AC12BF11BC12CF101011E512C5DDC
:1004500002E11D512B5D05E22B511D5F2C511E5BEE
:1004600003D001011D6B1E6B1FB716D01DC100F01C
:100470001EC101F0010E1D5F000E1E5B0050011039
:100480000BE00CC1E1FF0DC1E2FF200EE66E0C4B4C
:100490000D2B214B222BEAD72BC100F02CC101F0F0
:1004A000010E2B5F000E2C5B0050011013E029C1E0
:1004B000E9FF2AC1EAFFEECF00F00CC1E1FF0DC158
:1004C000E2FF00C0E6FF0C4B0D2B294B2A2B214BE2
:1004D000222BE2D71FA716D01DC100F01EC101F0CC
:1004E000010E1D5F000E1E5B005001100BE00CC1E1
:1004F000E1FF0DC1E2FF200EE66E0C4B0D2B214BF0
:10050000222BEAD793D511C1E9FF12C1EAFFEECF42
:1005100000F0EECF01F000C0E9FF01C0EAFFEECF2E
:100520001CF111C1E9FF12C1EAFFEECF00F0EECFDE
:1005300001F0020E0026000E012211C1E1FF12C1DE
:10054000E2FF00C0E6FF01C0E6FF1C0E296F010EAE
:100550002A6F010E2B6F000E2C6F6AD7C00E1F136F
:10056000000E20133BD01C51000AD8B40FD71C51E9
:100570006C0AD8B410D71C51660AD8B40ED71C51D7
:10058000450AD8B40CD71C51650AD8B409D71C51F8
:10059000670AD8B407D71C516F0AD8B405D71C51C5
:1005A000640AD8B403D71C51690AD8B4FFD61C51C9
:1005B000700AD8B4FCD61C51580AD8B4F8D61C51CD
:1005C000780AD8B4F5D61C51730AD8B4F3D61C51A6
:1005D000630A99E01C51750AC1E0B7D70101000E0A
:1005E0001F15006E2051070B016E00500110D8B48A
:1005F0007AEF0CF020A904D0060E1A6F000E1B6FC4
:1006000011C1E9FF12C1EAFFEECF00F0EECF01F019
:1006100000C0E9FF01C0EAFFEECF23F1EECF24F1E5
:10062000EECF25F1EECF26F111C1E9FF12C1EAFFAD
:10063000EECF00F0EECF01F0040E0026000E0122F6
:1006400011C1E1FF12C1E2FF00C0E6FF01C0E6FFF9
:10065000046A056A066A076A23C100F024C101F032
:1006600025C102F026C103F04FEC23F0010ED8B0F3
:10067000000E006E005206E00101257F030E1F13DD
:10068000000E20130101276B286B23C100F024C149
:1006900001F025C102F026C103F0046A056A066A6A
:1006A000076A64EC26F0000ED8A4010E006E00521A
:1006B000D8B49AD026C100F0016A026A036AFF0E1C
:1006C00000140101316F000E326F000E32177E0EE2
:1006D0002D6F000E2E6F2F6F306F2D51315D006E1C
:1006E0002E513259016E00C027F101C028F1010ED0
:1006F000005C276F000E0158286F27C100F028C149
:1007000001F0030E046E000E056E91EC25F000C0A2
:1007100027F101C028F10A0E046E000E056EB7EC39
:1007200023F000C027F101C028F1800E011801015B
:100730002D6F800E2D5D02E1000E005C04E2010EC3
:10074000275F000E285B010127510008006F49EC6C
:1007500011F023C104F024C105F025C106F026C123
:1007600007F0D8EC21F000C029F101C02AF102C045
:100770002BF103C02CF1000E046E000E056E000E6E
:10078000066E7F0E076E29C100F02AC101F02BC151
:1007900002F02CC103F04FEC23F0010ED8B0000E94
:1007A000006E005206E0010E0101275F000E285B7B
:1007B0001BD0000E046E000E056E200E066E820E1B
:1007C000076E29C100F02AC101F02BC102F02CC133
:1007D00003F04FEC23F0000ED8B0010E006E005273
:1007E00003E00101274B282B0101800E006E800ED3
:1007F00001012819005C02E12751000803E3010E02
:100800001C6F03D0010127C11CF120B11AD020A315
:1008100015D0800E2819006E7F0E005C02E1FC0EE0
:10082000275D0AE3800E2819006E800E1B19005CFC
:1008300002E11A51275D02E3010103D0010166EFD5
:1008400008F001011A511B1106E020A304D0010E8B
:100850001A5F000E1B5B000E006E1B51005C02E174
:100860001A51080803E2080E1C6F03D001011AC1D7
:100870001CF123C100F024C101F025C102F026C102
:1008800003F0046A056A066A076A64EC26F0000E43
:10089000D8A4010E006E0052D8B464D127C100F173
:1008A00049EC11F000C004F001C005F002C006F0F0
:1008B00003C007F023C100F024C101F025C102F0FC
:1008C00026C103F063EC1FF000C023F101C024F146
:1008D00002C025F103C026F101011C510008006F80
:1008E00049EC11F000C004F001C005F002C006F0B0
:1008F00003C007F023C100F024C101F025C102F0BC
:1009000026C103F063EC1FF000C02DF101C02EF1F1
:1009100002C02FF103C030F12DC123F12EC124F10B
:100920002FC125F130C126F12DC100F02EC101F0FB
:100930002FC102F030C103F00DEC20F0AAEC26F03C
:1009400000C004F001C005F002C006F003C007F0CB
:100950002DC100F02EC101F02FC102F030C103F013
:1009600031EC27F0000E046E000E056E000E066ED0
:100970007E0E076E4FEC23F0000ED8B0010E006E15
:1009800000521AE023C100F024C101F025C102F099
:1009900026C103F0000E046E000E056E000E066EFA
:1009A0007E0E076E31EC17F000C023F101C024F178
:1009B00002C025F103C026F123C100F024C101F0DB
:1009C00025C102F026C103F00DEC20F000C031F18A
:1009D00001C032F102C033F103C034F101011C51F6
:1009E000010F006E016A000E0122020E046E000E5D
:1009F00001BEFF0E026E036E0450010107E00036D7
:100A00000090013602360336FF0FF7D70101E20EE0
:100A100000264E0E0122000E022200C0F6FF01C089
:100A2000F7FF02C0F8FF0900F5CF2DF10900F5CF5F
:100A30002EF10900F5CF2FF10900F5CF30F130513B
:100A4000345D08E12F51335D05E12E51325D02E145
:100A50002D51315D1EE323C100F024C101F025C1F9
:100A600002F026C103F0CD0E046ECC0E056E4C0EC6
:100A7000066E7B0E076ED8EC21F000C023F101C09A
:100A800024F102C025F103C026F10101274B282BD8
:100A900069D0010123C100F024C101F025C102F099
:100AA00026C103F00DEC20F000C031F101C032F19D
:100AB00002C033F103C034F1020E046E1CC100F019
:100AC000000E016E026E036E0450000107E0003656
:100AD0000090013602360336FF0FF7D7E20E0026EC
:100AE0004E0E0122000E022200C0F6FF01C0F7FFE9
:100AF00002C0F8FF0900F5CF2DF10900F5CF2EF166
:100B00000900F5CF2FF10900F5CF30F10101305187
:100B1000345D08E12F51335D05E12E51325D02E174
:100B20002D51315D1FE223C100F024C101F025C128
:100B300002F026C103F0000E046E000E056E200EBA
:100B4000066E820E076ED8EC21F000C023F101C0C2
:100B500024F102C025F103C026F1010E0101275F37
:100B6000000E285B0101010120A398D020B796D088
:100B7000800E000A006E800E1B19005C02E11A5103
:100B80000A0804E20A0E1A6F000E1B6F010123C14E
:100B900000F024C101F025C102F026C103F00DECE4
:100BA00020F000C029F101C02AF102C02BF103C0DE
:100BB0002CF1010129512A112B112C1144E00A0EAC
:100BC000046E000E056E066E076E29C100F02AC184
:100BD00001F02BC102F02CC103F0D8EC1AF008C0D0
:100BE00000F009C001F00AC002F00BC003F0000ED3
:100BF00001012D6F031808E12D51021805E12D5157
:100C0000011802E10050000A1EE1010E01011A5F05
:100C1000000E1B5B0A0E046E000E056E066E076E5C
:100C200029C100F02AC101F02BC102F02CC103F050
:100C3000D8EC1AF000C029F101C02AF102C02BF152
:100C400003C02CF1B6D7800E01011B19006E800E77
:100C5000005C02E11C511A5D21E21A511C5D006F1B
:100C600049EC11F000C004F001C005F002C006F02C
:100C700003C007F023C100F024C101F025C102F038
:100C800026C103F063EC1FF000C023F101C024F182
:100C900002C025F103C026F11AC11CF10001050EA6
:100CA00001011A25006E000E1B21016E00501D5F10
:100CB00001501E5B1A511B1102E120A704D0010E46
:100CC0001D5F000E1E5B030E1F15006E20C101F09C
:100CD000000E01160050011004E0010E1D5F000E11
:100CE0001E5B1FA54AD01FA31AD0010E1F15006E50
:100CF00020C101F0000E01160050011003E02D0E7E
:100D0000006E02D02B0E006E0CC1E1FF0DC1E2FFA0
:100D100000C0E6FF0C4B0D2B214B222B14D0010EF3
:100D20001F15006E20C101F0000E011600500110C9
:100D30000AE00CC1E1FF0DC1E2FF200EE66E0C4B94
:100D40000D2B214B222B800E006E800E1E19005C95
:100D500002E11D5100080FE20CC1E1FF0DC1E2FFED
:100D6000300EE66E0C4B0D2B214B222B010E1D5F1E
:100D7000000E1E5BE8D701014BD01FB718D0800EC4
:100D8000006E800E1E19005C02E11D5100080FE28A
:100D90000CC1E1FF0DC1E2FF200EE66E0C4B0D2BE6
:100DA000214B222B010E1D5F000E1E5BE8D70101B7
:100DB0001FA31AD0010E1F15006E20C101F0000EF6
:100DC00001160050011003E02D0E006E02D02B0E14
:100DD000006E0CC1E1FF0DC1E2FF00C0E6FF0C4B4D
:100DE0000D2B214B222B14D0010E1F15006E20C19C
:100DF00001F0000E0116005001100AE00CC1E1FFE5
:100E00000DC1E2FF200EE66E0C4B0D2B214B222B69
:100E1000010123C100F024C101F025C102F026C167
:100E200003F00DEC20F000C029F101C02AF102C04E
:100E30002BF103C02CF1020E046E1CC100F0000E59
:100E4000016E026E036E0450000107E00036009050
:100E5000013602360336FF0FF7D7E20E00264E0E9C
:100E60000122000E022200C0F6FF01C0F7FF02C0FF
:100E7000F8FF0900F5CF04F00900F5CF05F00900EF
:100E8000F5CF06F00900F5CF07F029C100F02AC11F
:100E900001F02BC102F02CC103F0D8EC1AF0300E97
:100EA00000260CC1E1FF0DC1E2FF00C0E6FF010119
:100EB0000C4B0D2B214B222B1A511B1102E120A7A9
:100EC00076D00CC1E1FF0DC1E2FF2E0EE66E0101EE
:100ED0000C4B0D2B214B222B1C511A5F000E1B5B60
:100EE0001C5353E01C07020E046E1CC100F0000EE0
:100EF000016E026E036E0450010107E0003600909F
:100F0000013602360336FF0FF7D7E20E00264E0EEB
:100F10000122000E022200C0F6FF01C0F7FF02C04E
:100F2000F8FF0900F5CF04F00900F5CF05F009003E
:100F3000F5CF06F00900F5CF07F029C100F02AC16E
:100F400001F02BC102F02CC103F0D8EC1AF00A0E0C
:100F5000046E000E056E066E076ED8EC1AF008C01F
:100F600000F009C001F00AC002F00BC003F0300E1F
:100F700000260CC1E1FF0DC1E2FF00C0E6FF010148
:100F80000C4B0D2B214B222BABD71A511B110FE011
:100F90000CC1E1FF0DC1E2FF300EE66E0C4B0D2BD4
:100FA000214B222B010E1A5F000E1B5BEED71FABED
:100FB0000BD00CC1E1FF0DC1E2FF450EE66E0C4BFC
:100FC0000D2B214B222B0AD00CC1E1FF0DC1E2FFFA
:100FD000650EE66E0C4B0D2B214B222B800E281933
:100FE000006E800E005C02E1000E275D12E22751C8
:100FF0000008276F28C128F1E86A28570CC1E1FFD3
:101000000DC1E2FF2D0EE66E0C4B0D2B214B222B5A
:101010000BD001010CC1E1FF0DC1E2FF2B0EE66E0A
:101020000C4B0D2B214B222B0A0E046E000E056E6D
:1010300027C100F028C101F0B7EC23F0300E0026E4
:101040000CC1E1FF0DC1E2FF00C0E6FF01010C4B46
:101050000D2B214B222B0A0E046E000E056E27C1AC
:1010600000F028C101F0B7EC23F008C000F009C07F
:1010700001F0300E00260CC1E1FF0DC1E2FF00C0FF
:10108000E6FF01010C4B0D2B214B222B1FA71BD080
:10109000800E006E800E1E19005C02E11D510008DA
:1010A00012E20CC1E1FF0DC1E2FF200EE66E01016C
:1010B0000C4B0D2B214B222B010E1D5F000E1E5BD6
:1010C0001D511E11EEE1010116EF00F0010120A3F8
:1010D000FDD0800E2819006E800E005C02E1000E2B
:1010E000275D0AE2010E275D006E000E2859016E91
:1010F00000501A5F01501B5B23C100F024C101F0B6
:1011000025C102F026C103F00DEC20F000C029F14A
:1011100001C02AF102C02BF103C02CF1010E010124
:101120001C6F1C510A0A39E0020E046E1CC100F04B
:10113000000E016E026E036E0450010107E00036DE
:101140000090013602360336FF0FF7D70101E20E99
:1011500000264E0E0122000E022200C0F6FF01C042
:10116000F7FF02C0F8FF0900F5CF2DF10900F5CF18
:101170002EF10900F5CF2FF10900F5CF30F13051F4
:101180002C5D08E12F512B5D05E12E512A5D02E116
:101190002D51295D02E31C2BC4D701011C511A5D9E
:1011A000316F000E1B59326F31C11AF132C11BF180
:1011B00029C100F02AC101F02BC102F02CC103F0BB
:1011C000AAEC26F000C004F001C005F002C006F051
:1011D00003C007F023C100F024C101F025C102F0D3
:1011E00026C103F031EC27F000C02DF101C02EF133
:1011F00002C02FF103C030F131C100F149EC11F010
:101200002DC104F02EC105F02FC106F030C107F04A
:10121000D8EC21F0000E046E000E056E000E066E76
:101220007E0E076E31EC17F00DEC20F000C029F1B6
:1012300001C02AF102C02BF103C02CF101011A51A7
:101240001B1144E00A0E046E000E056E066E076E5A
:1012500029C100F02AC101F02BC102F02CC103F01A
:10126000D8EC1AF008C000F009C001F00AC002F082
:101270000BC003F0000E01012D6F031808E12D5182
:10128000021805E12D51011802E10050000A1EE18B
:101290000A0E046E000E056E066E076E29C100F080
:1012A0002AC101F02BC102F02CC103F0D8EC1AF0D6
:1012B00000C029F101C02AF102C02BF103C02CF1BA
:1012C000010E01011A5F000E1B5BB8D70101800EF1
:1012D000006E800E01011B19005C02E11A510C081E
:1012E00016E31AC100F145EC19F023C104F024C142
:1012F00005F025C106F026C107F031EC17F000C05B
:1013000023F101C024F102C025F103C026F123C15D
:1013100000F024C101F025C102F026C103F0046AE7
:10132000056A066A076A64EC26F0000ED8A4010E6E
:10133000006E0052D8B478D023C100F024C101F06F
:1013400025C102F026C103F00DEC20F0000E0101D2
:101350002D6F031808E12D51021805E12D510118D8
:1013600002E10050000A60E1800E006E800E281934
:10137000005C02E12751010857E227C100F149EC66
:1013800011F000C004F001C005F002C006F003C077
:1013900007F023C100F024C101F025C102F026C1ED
:1013A00003F063EC1FF05F0E046E700E056E090E05
:1013B000066E810E076E4FEC23F0010ED8B0000EC2
:1013C000006E005206E0090E0101275F000E285B47
:1013D00005D0080E0101275F000E285B27C100F130
:1013E00049EC11F000C004F001C005F002C006F0A5
:1013F00003C007F023C100F024C101F025C102F0B1
:1014000026C103F063EC1FF00DEC20F000C029F1C1
:1014100001C02AF102C02BF103C02CF10101236BA2
:10142000246B256B266B39D023C100F024C101F059
:1014300025C102F026C103F00DEC20F000C029F117
:1014400001C02AF102C02BF103C02CF129C100F028
:101450002AC101F02BC102F02CC103F0AAEC26F046
:1014600000C004F001C005F002C006F003C007F0A0
:1014700023C100F024C101F025C102F026C103F010
:1014800031EC27F000C023F101C024F102C025F1A6
:1014900003C026F10101276B286B010E1C6F1C5144
:1014A0000A0A39E0020E046E1CC100F0000E016E43
:1014B000026E036E0450010107E000360090013611
:1014C00002360336FF0FF7D70101E20E00264E0E5B
:1014D0000122000E022200C0F6FF01C0F7FF02C089
:1014E000F8FF0900F5CF2DF10900F5CF2EF1090025
:1014F000F5CF2FF10900F5CF30F130512C5D08E127
:101500002F512B5D05E12E512A5D02E12D51295D00
:1015100002E31C2BC4D701011C511A25006E000EDA
:101520001B21016E275100262851012200501D5F0A
:1015300001501E5B20B703D01A511B1104E0010EAD
:101540001D5F000E1E5B030E1F15006E20C101F013
:10155000000E01160050011004E0010E1D5F000E88
:101560001E5B1FA54AD01FA31AD0010E1F15006EC7
:1015700020C101F0000E01160050011003E02D0EF5
:10158000006E02D02B0E006E0CC1E1FF0DC1E2FF18
:1015900000C0E6FF0C4B0D2B214B222B14D0010E6B
:1015A0001F15006E20C101F0000E01160050011041
:1015B0000AE00CC1E1FF0DC1E2FF200EE66E0C4B0C
:1015C0000D2B214B222B800E006E800E1E19005C0D
:1015D00002E11D5100080FE20CC1E1FF0DC1E2FF65
:1015E000300EE66E0C4B0D2B214B222B010E1D5F96
:1015F000000E1E5BE8D701014BD01FB718D0800E3C
:10160000006E800E1E19005C02E11D5100080FE201
:101610000CC1E1FF0DC1E2FF200EE66E0C4B0D2B5D
:10162000214B222B010E1D5F000E1E5BE8D701012E
:101630001FA31AD0010E1F15006E20C101F0000E6D
:1016400001160050011003E02D0E006E02D02B0E8B
:10165000006E0CC1E1FF0DC1E2FF00C0E6FF0C4BC4
:101660000D2B214B222B14D0010E1F15006E20C113
:1016700001F0000E0116005001100AE00CC1E1FF5C
:101680000DC1E2FF200EE66E0C4B0D2B214B222BE1
:1016900001011CC100F01C07005252E0020E046E52
:1016A0001CC100F0000E016E026E036E04500101B9
:1016B00007E000360090013602360336FF0FF7D7F9
:1016C000E20E00264E0E0122000E022200C0F6FF9E
:1016D00001C0F7FF02C0F8FF0900F5CF04F00900D0
:1016E000F5CF05F00900F5CF06F00900F5CF07F0BA
:1016F00029C100F02AC101F02BC102F02CC103F076
:10170000D8EC1AF00A0E046E000E056E066E076E17
:10171000D8EC1AF008C000F009C001F00AC002F0CD
:101720000BC003F0300E00260CC1E1FF0DC1E2FF3B
:1017300000C0E6FF01010C4B0D2B214B222BA8D73B
:10174000800E006E800E2819005C02E1275100080F
:101750000FE20CC1E1FF0DC1E2FF300EE66E0C4B53
:101760000D2B214B222B010E275F000E285BE8D7A3
:101770000101800E000A006E800E1B19005C02E160
:101780001A51080803E2080E1C6F03D001011AC1A8
:101790001CF11C511A5F000E1B5B1C5302E120A7B9
:1017A0000AD00CC1E1FF0DC1E2FF2E0EE66E0C4B1C
:1017B0000D2B214B222B1CC100F149EC11F023C150
:1017C00004F024C105F025C106F026C107F0D8ECCD
:1017D00021F0AAEC20F000C029F101C02AF102C0DA
:1017E0002BF103C02CF101011C5353E01C07020E26
:1017F000046E1CC100F0000E016E026E036E0450F8
:10180000010107E000360090013602360336FF0F73
:10181000F7D7E20E00264E0E0122000E022200C073
:10182000F6FF01C0F7FF02C0F8FF0900F5CF04F092
:101830000900F5CF05F00900F5CF06F00900F5CF56
:1018400007F029C100F02AC101F02BC102F02CC120
:1018500003F0D8EC1AF00A0E046E000E056E066E48
:10186000076ED8EC1AF008C000F009C001F00AC0F9
:1018700002F00BC003F0300E00260CC1E1FF0DC1D9
:10188000E2FF00C0E6FF01010C4B0D2B214B222B88
:10189000AAD71A511B110FE00CC1E1FF0DC1E2FFE5
:1018A000300EE66E0C4B0D2B214B222B010E1A5FD6
:1018B000000E1B5BEED71FA71AD0800E006E800EA5
:1018C0001E19005C02E11D51000811E20CC1E1FF8C
:1018D0000DC1E2FF200EE66E0C4B0D2B214B222B8F
:1018E000010E1D5F000E1E5B1D511E11EFE1010177
:1018F00016EF00F0C00E1F152D6F20C12EF1000E47
:101900002E17000E2E1902E1000E2D19D8A482D038
:101910001FA929D011C1E9FF12C1EAFFEECF00F0E3
:10192000EECF01F000C0E9FF01C0EAFFEECF29F1E0
:10193000EECF2AF1EECF2BF1EECF2CF111C1E9FF62
:1019400012C1EAFFEECF00F0EECF01F0040E002648
:10195000000E012211C1E1FF12C1E2FF00C0E6FF4B
:1019600001C0E6FF2ED011C1E9FF12C1EAFFEECFA0
:1019700000F0EECF01F000C0E9FF01C0EAFFEECFBA
:1019800029F1EECF2AF1000E2ABFFF0E2B6F2C6F2C
:10199000000E2ABFFF0E2B6F2C6F11C1E9FF12C181
:1019A000EAFFEECF00F0EECF01F0020E0026000EAF
:1019B000012211C1E1FF12C1E2FF00C0E6FF01C038
:1019C000E6FF800E2C19006E800E005C08E1000E10
:1019D0002B5D05E1000E2A5D02E1000E295D18E293
:1019E000030E1F13000E2013006A016A026A036AC5
:1019F0002951005E2A51015A2B51025A2C51035A87
:101A000000C029F101C02AF102C02BF103C02CF162
:101A1000010156D001011FA929D011C1E9FF12C14E
:101A2000EAFFEECF00F0EECF01F000C0E9FF01C009
:101A3000EAFFEECF29F1EECF2AF1EECF2BF1EECF78
:101A40002CF111C1E9FF12C1EAFFEECF00F0EECF99
:101A500001F0040E0026000E012211C1E1FF12C1A7
:101A6000E2FF00C0E6FF01C0E6FF2AD011C1E9FF96
:101A700012C1EAFFEECF00F0EECF01F000C0E9FFA7
:101A800001C0EAFFEECF29F1EECF2AF1000E2B6F55
:101A90002C6F000E2B6F2C6F11C1E9FF12C1EAFFF2
:101AA000EECF00F0EECF01F0020E0026000E012274
:101AB00011C1E1FF12C1E2FF00C0E6FF01C0E6FF75
:101AC0000101000E1B1902E1000E1A190FE1000EB0
:101AD000006E2C1908E100502B1905E100502A195D
:101AE00002E12951000A02E11A4B1B2B0101C00E31
:101AF0001F15006E00C031F1C0D0010E1C6F1C51CB
:101B00000A0A39E0020E046E1CC100F0000E016EDC
:101B1000026E036E0450010107E0003600900136AA
:101B200002360336FF0FF7D70101E20E00264E0EF4
:101B30000122000E022200C0F6FF01C0F7FF02C022
:101B4000F8FF0900F5CF2DF10900F5CF2EF10900BE
:101B5000F5CF2FF10900F5CF30F130512C5D08E1C0
:101B60002F512B5D05E12E512A5D02E12D51295D9A
:101B700002E31C2BC4D701018FD0010E1C6F1C5136
:101B8000080A39E0020E046E1CC100F0000E016E5E
:101B9000026E036E0450010107E00036009001362A
:101BA00002360336FF0FF7D701010A0E00264F0E4B
:101BB0000122000E022200C0F6FF01C0F7FF02C0A2
:101BC000F8FF0900F5CF2DF10900F5CF2EF109003E
:101BD000F5CF2FF10900F5CF30F130512C5D08E140
:101BE0002F512B5D05E12E512A5D02E12D51295D1A
:101BF00002E31C2BC4D701014FD0010E1C6F1C51F6
:101C00000C0A39E0020E046E1CC100F0000E016ED9
:101C1000026E036E0450010107E0003600900136A9
:101C200002360336FF0FF7D701012A0E00264F0EAA
:101C30000122000E022200C0F6FF01C0F7FF02C021
:101C4000F8FF0900F5CF2DF10900F5CF2EF10900BD
:101C5000F5CF2FF10900F5CF30F130512C5D08E1BF
:101C60002F512B5D05E12E512A5D02E12D51295D99
:101C700002E31C2BC4D701010FD03151000AD8B4A4
:101C80003CD73151C00AD8B438D73151800AD8B4C2
:101C900074D73151400AB1E00101800E006E800E10
:101CA0001B19005C02E11A511C5D03E21AC11CF110
:101CB0000ED00101800E1B19006E800E005C02E147
:101CC0001C511A5D04E21CC11AF1000E1B6F0101C8
:101CD00001011D511E110EE0030E1F15006E20C1E3
:101CE00001F0000E01160050011004E0010E1D5F0E
:101CF000000E1E5B800E1B19006E800E1E19005C0C
:101D000002E11D511A5D05E21A511D5F1B511E5B58
:101D100003D001011D6B1E6BC40E1F152D6F2051CA
:101D2000080B2E6F2E51080A02E1400E2D1908E112
:101D30001D511E1104E0010E1D5F000E1E5B1ED022
:101D40000101C00E1F152D6F2051080B2E6F2E5153
:101D5000080A02E1800E2D1911E1800E006E800E3E
:101D60001E19005C02E11D51020805E2020E1D5F12
:101D7000000E1E5B03D001011D6B1E6B01010101F2
:101D80001FA56ED01FA31AD0010E1F15006E20C113
:101D900001F0000E01160050011003E02D0E006E40
:101DA00002D02B0E006E0CC1E1FF0DC1E2FF00C09E
:101DB000E6FF0C4B0D2B214B222B3CD0010E1F15A7
:101DC000006E20C101F0000E0116005001100BE062
:101DD0000CC1E1FF0DC1E2FF200EE66E0C4B0D2B96
:101DE000214B222B27D0C00E1F152D6F2051080B21
:101DF0002E6F2E51080A02E1800E2D191BE10CC135
:101E0000E1FF0DC1E2FF300EE66E0C4B0D2B214BB6
:101E1000222B1FAB03D0580E006E02D0780E006E3E
:101E20000CC1E1FF0DC1E2FF00C0E6FF0C4B0D2B22
:101E3000214B222B01011D511E1111E00CC1E1FFAC
:101E40000DC1E2FF300EE66E0C4B0D2B214B222B09
:101E5000010E1D5F000E1E5B1D511E11EFE185D0AE
:101E60001D511E1113E01FB711D00CC1E1FF0DC1B0
:101E7000E2FF200EE66E0C4B0D2B214B222B010EA8
:101E80001D5F000E1E5B1D511E11EFE11FA31AD036
:101E9000010E1F15006E20C101F0000E011600504A
:101EA000011003E02D0E006E02D02B0E006E0CC14F
:101EB000E1FF0DC1E2FF00C0E6FF0C4B0D2B214BF3
:101EC000222B14D0010E1F15006E20C101F0000E50
:101ED0000116005001100AE00CC1E1FF0DC1E2FF44
:101EE000200EE66E0C4B0D2B214B222BC00E1F1526
:101EF0002D6F2051080B2E6F2E51080A02E1400E63
:101F00002D190BE10CC1E1FF0DC1E2FF300EE66EB1
:101F10000C4B0D2B214B222B28D00101C00E1F157D
:101F20002D6F2051080B2E6F2E51080A02E1800EF2
:101F30002D191BE10CC1E1FF0DC1E2FF300EE66E71
:101F40000C4B0D2B214B222B1FAB03D0580E006ED8
:101F500002D0780E006E0CC1E1FF0DC1E2FF00C09F
:101F6000E6FF0C4B0D2B214B222B01010101800EB2
:101F7000006E800E1B19005C02E11A511C5D0BE221
:101F80000CC1E1FF0DC1E2FF300EE66E0C4B0D2BD4
:101F9000214B222BEAD701011AC100F01BC101F02D
:101FA000010E1A5F000E1B5B00500110D8B44DD11A
:101FB000C00E1F15006E00C02DF12BD1020E046E55
:101FC0001AC100F01BC101F0000E1BBFFF0E026E14
:101FD000036E0450010107E000360090013602361E
:101FE0000336FF0FF7D7E20E00264E0E0122000E39
:101FF000022200C0F6FF01C0F7FF02C0F8FF09008F
:10200000F5CF04F00900F5CF05F00900F5CF06F093
:102010000900F5CF07F029C100F02AC101F02BC15A
:1020200002F02CC103F0D8EC1AF00A0E046E000E78
:10203000056E066E076ED8EC1AF008C000F009C0F5
:1020400001F00AC002F00BC003F0300E00240101C1
:102050001C6FEFD01FAB4ED0020E046E1AC100F001
:102060001BC101F0000E1BBFFF0E026E036E045079
:10207000010107E000360090013602360336FF0FFB
:10208000F7D701010A0E00264F0E0122000E022290
:1020900000C0F6FF01C0F7FF02C0F8FF0900F5CF4E
:1020A00004F00900F5CF05F00900F5CF06F00900AE
:1020B000F5CF07F029C100F02AC101F02BC102F0D1
:1020C0002CC103F0D8EC1AF00F0E0016000E01160A
:1020D000021603165A0E00264F0E0122000E02228F
:1020E00000C0F6FF01C0F7FF02C0F8FF0900F5CFFE
:1020F0001CF14ED0020E046E1AC100F01BC101F09B
:10210000000E01011BBFFF0E026E036E04500101A1
:1021100007E000360090013602360336FF0FF7D78E
:1021200001010A0E00264F0E0122000E022200C0FD
:10213000F6FF01C0F7FF02C0F8FF0900F5CF04F079
:102140000900F5CF05F00900F5CF06F00900F5CF3D
:1021500007F029C100F02AC101F02BC102F02CC107
:1021600003F0D8EC1AF00F0E0016000E011602163E
:1021700003166C0E00264F0E0122000E022200C034
:10218000F6FF01C0F7FF02C0F8FF0900F5CF1CF110
:1021900000014FD0020E046E1AC100F01BC101F005
:1021A000000E01011BBFFF0E026E036E0450010101
:1021B00007E000360090013602360336FF0FF7D7EE
:1021C0002A0E00264F0E0122000E022200C0F6FF4A
:1021D00001C0F7FF02C0F8FF0900F5CF04F00900C5
:1021E000F5CF05F00900F5CF06F00900F5CF07F0AF
:1021F00029C100F02AC101F02BC102F02CC103F06B
:10220000D8EC1AF0070E001401011C6F300E1C27C9
:1022100010D001012D51000AD8B4D0D62D51C00ADA
:10222000D8B4CCD62D51800AD8B414D72D51400A39
:10223000B1E001010CC1E1FF0DC1E2FF1CC1E6FFED
:102240000C4B0D2B214B222BA6D61FA71AD0800E8C
:10225000006E800E1E19005C02E11D51000811E2A3
:102260000CC1E1FF0DC1E2FF200EE66E0C4B0D2B01
:10227000214B222B010E1D5F000E1E5B1D511E11F6
:10228000EFE1010116EF00F021C100F022C101F0E1
:102290001200800E01010019006E800E000A005C21
:1022A000D8B081D100510008046E04C000F1800E46
:1022B0000418006E800E6E0A005CD8A0C6D0640EB2
:1022C000046E00C100F01CEC24F0120E0026000E7B
:1022D00000BEFF0E016E000E0122020E046E000E03
:1022E00001BEFF0E026E036E0450000107E00036CF
:1022F0000090013602360336FF0FF7D700017A0E41
:1023000000264E0E0122000E022200C0F6FF01C080
:10231000F7FF02C0F8FF0900F5CF35F10900F5CF4E
:1023200036F10900F5CF37F10900F5CF38F1640E29
:10233000046E00C100F01CEC24F008C000F00A0E8E
:10234000046E1CEC24F0090E0026000E00BEFF0EE9
:10235000016E000E0122020E046E000E01BEFF0E81
:10236000026E036E0450000107E000360090013653
:1023700002360336FF0FF7D700017A0E00264E0E05
:102380000122000E022200C0F6FF01C0F7FF02C0CA
:10239000F8FF0900F5CF00F00900F5CF01F00900C2
:1023A000F5CF02F00900F5CF03F035C104F036C1D6
:1023B00005F037C106F038C107F0D8EC21F000C0B5
:1023C00035F101C036F102C037F103C038F10A0E11
:1023D000046E00C100F01CEC24F008C000F0020EF6
:1023E000046E000E00BEFF0E016E026E036E0450FE
:1023F000000107E000360090013602360336FF0F79
:10240000F7D700017A0E00264E0E0122000E02229E
:1024100000C0F6FF01C0F7FF02C0F8FF0900F5CFCA
:1024200000F00900F5CF01F00900F5CF02F0090036
:10243000F5CF03F035C104F036C105F037C106F021
:1024400038C107F0D8EC21F01200800E0A0A006EA5
:10245000800E01010019005C76E20A0E046E00C1D4
:1024600000F01CEC24F0090E0026000E00BEFF0E4A
:10247000016E000E0122020E046E000E01BEFF0E60
:10248000026E036E0450000107E000360090013632
:1024900002360336FF0FF7D700017A0E00264E0EE4
:1024A0000122000E022200C0F6FF01C0F7FF02C0A9
:1024B000F8FF0900F5CF35F10900F5CF36F1090035
:1024C000F5CF37F10900F5CF38F10A0E046E00C1DF
:1024D00000F01CEC24F008C000F0020E046E000EA8
:1024E00000BEFF0E016E026E036E0450000107E095
:1024F00000360090013602360336FF0FF7D7000191
:102500007A0E00264E0E0122000E022200C0F6FFB7
:1025100001C0F7FF02C0F8FF0900F5CF00F0090085
:10252000F5CF01F00900F5CF02F00900F5CF03F077
:1025300035C104F036C105F037C106F038C107F0E7
:10254000D8EC21F012000001020E046E00C100F070
:10255000000E010100BFFF0E016E026E036E0450FB
:10256000010107E000360090013602360336FF0F06
:10257000F7D701017A0E00264E0E0122000E02222C
:1025800000C0F6FF01C0F7FF02C0F8FF0900F5CF59
:1025900000F00900F5CF01F00900F5CF02F00900C5
:1025A000F5CF03F01200800E0019006E800E6E0A47
:1025B000005CD8A0C6D0640E046E00C100F01CEC14
:1025C00024F0120E0026000E00BEFF0E016E000E5B
:1025D0000122020E046E000E01BEFF0E026E036E9B
:1025E0000450000107E00036009001360236033641
:1025F000FF0FF7D70001AE0E00264E0E0122000E8F
:10260000022200C0F6FF01C0F7FF02C0F8FF090078
:10261000F5CF35F10900F5CF36F10900F5CF37F1E7
:102620000900F5CF38F1640E046E00C100F01CEC17
:1026300024F008C000F00A0E046E1CEC24F0090E11
:102640000026000E00BEFF0E016E000E0122020EDB
:10265000046E000E01BEFF0E026E036E04500001F8
:1026600007E000360090013602360336FF0FF7D739
:102670000001AE0E00264E0E0122000E022200C006
:10268000F6FF01C0F7FF02C0F8FF0900F5CF00F028
:102690000900F5CF01F00900F5CF02F00900F5CFF0
:1026A00003F035C104F036C105F037C106F038C17A
:1026B00007F0D8EC21F000C035F101C036F102C0BE
:1026C00037F103C038F10A0E046E00C100F01CECB3
:1026D00024F008C000F0020E046E000E00BEFF0ED3
:1026E000016E026E036E0450000107E00036009098
:1026F000013602360336FF0FF7D70001AE0E002673
:102700004E0E0122000E022200C0F6FF01C0F7FFAC
:1027100002C0F8FF0900F5CF00F00900F5CF01F085
:102720000900F5CF02F00900F5CF03F035C104F040
:1027300036C105F037C106F038C107F0D8EC21F0FA
:102740001200800E0A0A006E800E01010019005C62
:1027500076E20A0E046E00C100F01CEC24F0090EB3
:102760000026000E00BEFF0E016E000E0122020EBA
:10277000046E000E01BEFF0E026E036E04500001D7
:1027800007E000360090013602360336FF0FF7D718
:102790000001AE0E00264E0E0122000E022200C0E5
:1027A000F6FF01C0F7FF02C0F8FF0900F5CF35F1D1
:1027B0000900F5CF36F10900F5CF37F10900F5CF63
:1027C00038F10A0E046E00C100F01CEC24F008C0C1
:1027D00000F0020E046E000E00BEFF0E016E026ECF
:1027E000036E0450000107E0003600900136023607
:1027F0000336FF0FF7D70001AE0E00264E0E012262
:10280000000E022200C0F6FF01C0F7FF02C0F8FF71
:102810000900F5CF00F00900F5CF01F00900F5CF70
:1028200002F00900F5CF03F035C104F036C105F020
:1028300037C106F038C107F0D8EC21F012000001D2
:10284000020E046E00C100F0000E010100BFFF0E79
:10285000016E026E036E0450010107E00036009025
:10286000013602360336FF0FF7D7AE0E00264E0EA6
:102870000122000E022200C0F6FF01C0F7FF02C0D5
:10288000F8FF0900F5CF00F00900F5CF01F00900CD
:10289000F5CF02F00900F5CF03F01200200E000181
:1028A000BC6F200EBD6FBE6BE06BE16BE26BE36B48
:1028B000E46BE56BE66BE76BE86BE96BEA6BEB6B84
:1028C000EC6BED6BEE6BEF6B010EF86F0F0EF96FAB
:1028D000BC0EFA6F000EFB6FC4EC24F0820E0B6E80
:1028E000FF0E0A6E0B2E01D003D00A2EFED7FAD7A8
:1028F000870E0A6E0A2EFED70000BF6B200EBF5D4A
:10290000D8B034D1020E046EBFC0F4F0000EF56FE3
:10291000F66FF76F045007E0F437F491F537F637A8
:10292000F737FF0FF8D700017E0EF425006E4F0E2B
:10293000F521016E000EF621026E000E00C0F6FFBA
:1029400001C0F7FF02C0F8FF0900F5CF04F009004D
:10295000F5CF05F00900F5CF06F00900F5CF07F037
:102960001A0EF425E96E000EF521EA6EEECF00F0A6
:10297000EECF01F0EECF02F0EECF03F0D8EC21F075
:10298000520E046EB80E056E1E0E066E7D0E076E9C
:10299000D8EC21F0E0C004F0E1C005F0E2C006F0A0
:1029A000E3C007F031EC17F000C0E0F001C0E1F047
:1029B00002C0E2F003C0E3F0FE0EF425006E4F0EFD
:1029C000F521016E000EF621026E000E00C0F6FF2A
:1029D00001C0F7FF02C0F8FF0900F5CF04F00900BD
:1029E000F5CF05F00900F5CF06F00900F5CF07F0A7
:1029F0001A0EF425E96E000EF521EA6EEECF00F016
:102A0000EECF01F0EECF02F0EECF03F0D8EC21F0E4
:102A1000520E046EB80E056E1E0E066E7D0E076E0B
:102A2000D8EC21F0E4C004F0E5C005F0E6C006F003
:102A3000E7C007F031EC17F000C0E4F001C0E5F0AA
:102A400002C0E6F003C0E7F07E0EF425006E500EE3
:102A5000F521016E000EF621026E000E00C0F6FF99
:102A600001C0F7FF02C0F8FF0900F5CF04F009002C
:102A7000F5CF05F00900F5CF06F00900F5CF07F016
:102A80001A0EF425E96E000EF521EA6EEECF00F085
:102A9000EECF01F0EECF02F0EECF03F0D8EC21F054
:102AA000520E046EB80E056E1E0E066E7D0E076E7B
:102AB000D8EC21F0E8C004F0E9C005F0EAC006F067
:102AC000EBC007F031EC17F000C0E8F001C0E9F00E
:102AD00002C0EAF003C0EBF0FE0EF425006E500ECB
:102AE000F521016E000EF621026E000E00C0F6FF09
:102AF00001C0F7FF02C0F8FF0900F5CF04F009009C
:102B0000F5CF05F00900F5CF06F00900F5CF07F085
:102B10001A0EF425E96E000EF521EA6EEECF00F0F4
:102B2000EECF01F0EECF02F0EECF03F0D8EC21F0C3
:102B3000520E046EB80E056E1E0E066E7D0E076EEA
:102B4000D8EC21F0ECC004F0EDC005F0EEC006F0CA
:102B5000EFC007F031EC17F000C0ECF001C0EDF071
:102B600002C0EEF003C0EFF0BF2BC8D6E0C000F00B
:102B7000E1C001F0E2C002F0E3C003F0E0C004F005
:102B8000E1C005F0E2C006F0E3C007F0D8EC21F0A8
:102B900000C0F4F001C0F5F002C0F6F003C0F7F099
:102BA000E4C000F0E5C001F0E6C002F0E7C003F0C9
:102BB000E4C004F0E5C005F0E6C006F0E7C007F0A9
:102BC000D8EC21F0F4C004F0F5C005F0F6C006F032
:102BD000F7C007F031EC17F000C0F8F001C0F9F0D1
:102BE00002C0FAF003C0FBF062EC1CF000C0E0F0A1
:102BF00001C0E1F002C0E2F003C0E3F0000E046E99
:102C0000000E056E000E066E7B0E076ED8EC21F0EE
:102C100000C0E0F001C0E1F002C0E2F003C0E3F068
:102C2000E8C000F0E9C001F0EAC002F0EBC003F038
:102C3000E8C004F0E9C005F0EAC006F0EBC007F018
:102C4000D8EC21F000C0F4F001C0F5F002C0F6F0BD
:102C500003C0F7F0ECC000F0EDC001F0EEC002F0F0
:102C6000EFC003F0ECC004F0EDC005F0EEC006F0DC
:102C7000EFC007F0D8EC21F0F4C004F0F5C005F087
:102C8000F6C006F0F7C007F031EC17F000C0F8F01E
:102C900001C0F9F002C0FAF003C0FBF062EC1CF0D6
:102CA00000C0E8F001C0E9F002C0EAF003C0EBF0B8
:102CB000000E046E000E056E000E066E7B0E076E93
:102CC000D8EC21F000C0E8F001C0E9F002C0EAF061
:102CD00003C0EBF0000E046E000E056E480E066E8B
:102CE000850E076ED8EC21F0E0C004F0E1C005F0DD
:102CF000E2C006F0E3C007F063EC1FF000C0F0F0A4
:102D000001C0F1F002C0F2F003C0F3F000C004F023
:102D100001C005F002C006F003C007F0000E006E0F
:102D2000000E016E200E026E810E036E4FEC23F03A
:102D3000010ED8B0000E006E005218E1000E046EB5
:102D4000000E056E200E066E830E076EE0C000F0CA
:102D5000E1C001F0E2C002F0E3C003F04FEC23F069
:102D6000010ED8B0000E006E00520EE00001829EEF
:102D7000046A82BE042A000E04B0400E8218400B82
:102D8000821A010E186E0CD00001828E046A82BE77
:102D9000042A000E04B0400E8218400B821A186AF2
:102DA000C00E0101016F000E026F7E0E036F510E07
:102DB000046F000E056FE0C006F1E1C007F1E2C04C
:102DC00008F1E3C009F121EC26F0800E006F77ECEA
:102DD00024F0C00E0001F86F000EF96F48EC26F0E9
:102DE000C00E0101016F000E026F880E036F510EBD
:102DF000046F000E056FE8C006F1E9C007F1EAC0F4
:102E000008F1EBC009F121EC26F0C00E006F77EC61
:102E100024F0C00E0001F86F000EF96F48EC26F0A8
:102E2000C00E0101016F000E026F920E036F510E72
:102E3000046F000E056FF0C006F1F1C007F1F2C09B
:102E400008F1F3C009F121EC26F0020E0001F86F41
:102E5000090EF96FC00EFA6F000EFB6FC4EC24F080
:102E600012000001025006180E6E086A096A0B6A09
:102E70000350076425EF18F006500A6E068E028E86
:102E800003500B6E0750036E000E0B6475EF17F0C6
:102E90000B50075ED8B416EF18F0070E0764E4EF86
:102EA00017F0075E00C008F001C000F002C001F09A
:102EB000026A074E16EF18F00764B9EF17F0075EC5
:102EC00000C008F001C000F0016A074E16EF18F0CC
:102ED000076497EF17F0075E00C008F0006A074E1E
:102EE00016EF18F007647EEF17F00AC002F005C075
:102EF00001F004C000F0086A42EF19F0030E076405
:102F000089EF17F0075E08380F0B086E074E16EFB3
:102F100018F0D8900832074E16EF18F0D890083203
:102F2000074E16EF18F0D890083216EF18F0030E7F
:102F30000764A8EF17F0075E08380F0B086E00381B
:102F4000F00B082600380F0B006E074E16EF18F036
:102F5000D89000320832074E16EF18F0D8900032A1
:102F60000832074E16EF18F0D8900032083216EFEC
:102F700018F0030E0764D0EF17F0075E08380F0B48
:102F8000086E0038F00B082600380F0B006E013871
:102F9000F00B002601380F0B016E074E16EF18F0EC
:102FA000D890013200320832074E16EF18F0D89050
:102FB000013200320832074E16EF18F0D890013275
:102FC0000032083216EF18F0030E076401EF18F014
:102FD000075E08380F0B086E0038F00B0826003823
:102FE0000F0B006E0138F00B002601380F0B016E3D
:102FF0000238F00B012602380F0B026E074E16EF57
:1030000018F0D8900232013200320832074E16EF23
:1030100018F0D8900232013200320832074E16EF13
:1030200018F0D8900232013200320832096A000EDC
:103030000EAE0AEF19F0081E001E011E021E082A1D
:103040000022012202220AEF19F00750D8A42BEF28
:1030500018F042EF19F0096A02C00AF0028E068EDB
:103060000750035C076ED8B4FDEF18F0070E076435
:10307000CBEF18F0075E0450096E0550046E065041
:10308000056E066A074EFDEF18F0070E0764A0EF05
:1030900018F0075E0450096E0550046E056A074E6D
:1030A000FDEF18F0070E07647EEF18F0075E04507E
:1030B000096E046A074EFDEF18F0070E076465EF0E
:1030C00018F00AC002F042EF19F0030E076470EF27
:1030D00018F0075E09380F0B096E074EFDEF18F068
:1030E000D8900932074EFDEF18F0D8900932074EFC
:1030F000FDEF18F0D8900932FDEF18F0030E0764C9
:103100008FEF18F0075E09380F0B096E0438F00BCB
:10311000092604380F0B046E074EFDEF18F0D89007
:1031200004320932074EFDEF18F0D890043209320C
:10313000074EFDEF18F0D89004320932FDEF18F079
:10314000030E0764B7EF18F0075E09380F0B096E1E
:103150000438F00B092604380F0B046E0538F00B09
:10316000042605380F0B056E074EFDEF18F0D890BA
:10317000053204320932074EFDEF18F0D8900532BF
:1031800004320932074EFDEF18F0D89005320432B0
:103190000932FDEF18F0030E0764E8EF18F0075E40
:1031A00009380F0B096E0438F00B092604380F0B91
:1031B000046E0538F00B042605380F0B056E063833
:1031C000F00B052606380F0B066E074EFDEF18F0C4
:1031D000D8900632053204320932074EFDEF18F05E
:1031E000D8900632053204320932074EFDEF18F04E
:1031F000D8900632053204320932086A000E0EAE4B
:103200000AEF19F0091E041E051E061E092A0422D3
:1032100005220622095008260450002205500122EA
:10322000065002220EBE21EF19F0D8A030EF19F09F
:103230000232013200320832033E30EF19F03CEF27
:1032400019F0D8B036EF19F0000E081E001E011E4E
:10325000021E082A0022012202220A7E36EF19F0FD
:10326000010E0C6E6DEC1EF044EF19F0020E0C6EA8
:103270006DEC1EF044EF19F0040E0C6E09EC27F013
:1032800044EF19F0000E0C6E12006E0E0101005D8D
:10329000D8A0D0D0640E046E00C100F0BEEC26F0C1
:1032A000120E0026016A000E0122020E046E000EAC
:1032B00001BEFF0E026E036E0450000107E00036EF
:1032C0000090013602360336FF0FF7D700017A0E61
:1032D00000264E0E0122000E022200C0F6FF01C0A1
:1032E000F7FF02C0F8FF0900F5CF00F00900F5CFA5
:1032F00001F00900F5CF02F00900F5CF03F0000E50
:10330000046E000E056E000E066E7E0E076ED8EC83
:1033100021F000C035F101C036F102C037F103C021
:1033200038F1640E046E00C100F0BEEC26F008C057
:1033300000F00A0E046EBEEC26F0090E0026016AAB
:10334000000E0122020E046E000E01BEFF0E026E80
:10335000036E0450000107E000360090013602368B
:103360000336FF0FF7D700017A0E00264E0E01221A
:10337000000E022200C0F6FF01C0F7FF02C0F8FFF6
:103380000900F5CF00F00900F5CF01F00900F5CFF5
:1033900002F00900F5CF03F035C104F036C105F0A5
:1033A00037C106F038C107F0D8EC21F000C035F184
:1033B00001C036F102C037F103C038F10A0E046EC5
:1033C00000C100F0BEEC26F008C000F0020E046E52
:1033D000000E016E026E036E0450000107E000361D
:1033E0000090013602360336FF0FF7D700017A0E40
:1033F00000264E0E0122000E022200C0F6FF01C080
:10340000F7FF02C0F8FF0900F5CF00F00900F5CF83
:1034100001F00900F5CF02F00900F5CF03F035C146
:1034200004F036C105F037C106F038C107F0D8EC1A
:1034300021F01200010100510A08D8B083D00A0E11
:10344000046E00C100F0BEEC26F0090E0026016AF1
:10345000000E0122020E046E000E01BEFF0E026E6F
:10346000036E0450000107E000360090013602367A
:103470000336FF0FF7D700017A0E00264E0E012209
:10348000000E022200C0F6FF01C0F7FF02C0F8FFE5
:103490000900F5CF00F00900F5CF01F00900F5CFE4
:1034A00002F00900F5CF03F0000E046E000E056E69
:1034B000000E066E7E0E076ED8EC21F000C035F1CE
:1034C00001C036F102C037F103C038F10A0E046EB4
:1034D00000C100F0BEEC26F008C000F0020E046E41
:1034E000000E016E026E036E0450000107E000360C
:1034F0000090013602360336FF0FF7D700017A0E2F
:1035000000264E0E0122000E022200C0F6FF01C06E
:10351000F7FF02C0F8FF0900F5CF00F00900F5CF72
:1035200001F00900F5CF02F00900F5CF03F035C135
:1035300004F036C105F037C106F038C107F0D8EC09
:1035400021F012000001020E046E00C100F0000E16
:10355000016E026E036E0450000107E00036009019
:10356000013602360336FF0FF7D77A0E00264E0ECD
:103570000122000E022200C0F6FF01C0F7FF02C0C8
:10358000F8FF0900F5CF00F00900F5CF01F00900C0
:10359000F5CF02F00900F5CF03F0000E046E000E27
:1035A000056E000E066E7E0E076ED8EC21F012003E
:1035B00000010B6A0A6A096A086A0E6A033408364F
:1035C0000450085E0550D8A0053C095E0650D8A0FE
:1035D000063C0A5E0750D8A0073C0B5EE86AD8A0FC
:1035E000010E0E5E0336070E0C6E033408360936E4
:1035F0000A360B360E36045003A012EF1BF0085E9D
:103600000550D8A0053C095E0650D8A0063C0A5ECD
:103610000750D8A0073C0B5EE86AD8A0010E0E5EEA
:1036200023EF1BF008260550D8B0053C09260650AC
:10363000D8B0063C0A260750D8B0073C0B26E86AEB
:10364000D8B0010E0E2603360C2EF5EF1AF0023418
:10365000083609360A360B360E36045003A044EFFE
:103660001BF0085E0550D8A0053C095E0650D8A0A6
:10367000063C0A5E0750D8A0073C0B5EE86AD8A05B
:10368000010E0E5E55EF1BF008260550D8B0053C24
:1036900009260650D8B0063C0A260750D8B0073C89
:1036A0000B26E86AD8B0010E0E260236070E0C6E05
:1036B0000234083609360A360B360E36045002A09C
:1036C00075EF1BF0085E0550D8A0053C095E06505A
:1036D000D8A0063C0A5E0750D8A0073C0B5EE86AFB
:1036E000D8A0010E0E5E86EF1BF008260550D8B05C
:1036F000053C09260650D8B0063C0A260750D8B02B
:10370000073C0B26E86AD8B0010E0E2602360C2EB6
:1037100058EF1BF00134083609360A360B360E36E0
:10372000045002A0A7EF1BF0085E0550D8A0053C8E
:10373000095E0650D8A0063C0A5E0750D8A0073C98
:103740000B5EE86AD8A0010E0E5EB8EF1BF00826EB
:103750000550D8B0053C09260650D8B0063C0A26CC
:103760000750D8B0073C0B26E86AD8B0010E0E26E9
:103770000136070E0C6E0134083609360A360B3650
:103780000E36045001A0D8EF1BF0085E0550D8A0FB
:10379000053C095E0650D8A0063C0A5E0750D8A03A
:1037A000073C0B5EE86AD8A0010E0E5EE9EF1BF045
:1037B00008260550D8B0053C09260650D8B0063C6E
:1037C0000A260750D8B0073C0B26E86AD8B0010E8D
:1037D0000E2601360C2EBBEF1BF0003408360936DE
:1037E0000A360B360E36045001A00AEF1CF0085EB4
:1037F0000550D8A0053C095E0650D8A0063C0A5EDC
:103800000750D8A0073C0B5EE86AD8A0010E0E5EF8
:103810001BEF1CF008260550D8B0053C09260650C1
:10382000D8B0063C0A260750D8B0073C0B26E86AF9
:10383000D8B0010E0E260036070E0C6E0034083686
:1038400009360A360B360E36045000A03BEF1CF04A
:10385000085E0550D8A0053C095E0650D8A0063C7D
:103860000A5E0750D8A0073C0B5EE86AD8A0010E9C
:103870000E5E4CEF1CF008260550D8B0053C09261A
:103880000650D8B0063C0A260750D8B0073C0B2695
:10389000E86AD8B0010E0E2600360C2E1EEF1CF082
:1038A00000B061EF1CF0045008260550D8B0053C6C
:1038B00009260650D8B0063C0A260750D8B0073C67
:1038C0000B261200F8C004F0F9C005F0FAC006F0AB
:1038D000FBC007F0006A016A026A036A4FEC23F03A
:1038E000000ED8B0010E006E005205E0006A016AB9
:1038F000026A036A12000001F8C001F1F9C002F186
:10390000FAC003F1FBC004F1000E046E000E056E58
:10391000000E066E7F0E076EF8C000F0F9C001F0D1
:10392000FAC002F0FBC003F04FEC23F0010ED8B058
:10393000000E006E00521AE001C104F002C105F051
:1039400003C106F004C107F0000E006E000E016E08
:10395000000E026E7F0E036E63EC1FF000C001F1DB
:1039600001C002F102C003F103C004F101C10CF176
:1039700002C10DF103C10EF104C10FF10A0E0101E4
:10398000106F010E116FF6EC25F000C001F101C0BF
:1039900002F102C003F103C004F100C00CF101C048
:1039A0000DF102C00EF103C00FF1020E046E000E05
:1039B000056E0AC100F00BC101F0B7EC23F000C0A6
:1039C00010F101C011F1E6EC22F000C001F101C0DC
:1039D00002F102C003F103C004F1000E046E000EF8
:1039E000056E000E066E7F0E076EF8C000F0F9C07F
:1039F00001F0FAC002F0FBC003F04FEC23F0010E1F
:103A0000D8B0000E006E00521AE001C104F002C1ED
:103A100005F003C106F004C107F0000E006E000EB1
:103A2000016E000E026E7F0E036E63EC1FF000C08D
:103A300001F101C002F102C003F103C004F1140E50
:103A40000101096F01C104F002C105F003C106F0D4
:103A500004C107F0F8C000F0F9C001F0FAC002F0AC
:103A6000FBC003F063EC1FF001C104F002C105F0DC
:103A700003C106F004C107F031EC17F0000E046E2C
:103A8000000E056E000E066E800E076E63EC1FF0D2
:103A900000C005F101C006F102C007F103C008F142
:103AA00001C104F002C105F003C106F004C107F032
:103AB00064EC26F0010ED8A4000E006E00520CE15A
:103AC00005C101F106C102F107C103F108C104F10A
:103AD000010109070953B6E101C100F002C101F07B
:103AE00003C102F004C103F012003E0E0001BC6FDE
:103AF0003C0EBD6FBE6B2D0EBF6F2D0EC06FC16B28
:103B00006F0EC26F760EC36FC46B200EC56F200E92
:103B1000C66FC76B18520BE0010EF86F0F0EF96FEE
:103B2000BC0EFA6F000EFB6FC4EC24F00AD0010E3D
:103B3000F86F0F0EF96FBF0EFA6F000EFB6FC4EC3B
:103B400024F0020E0C6EFF0E0B6EFF0E0A6E0C2E92
:103B500001D007D00B2E01D003D00A2EFED7FAD702
:103B6000F6D7060E0B6EFF0E0A6E0B2E01D003D099
:103B70000A2EFED7FAD70A0E0A6E0A2EFED719525F
:103B80000BE0010EF86F0A0EF96FC20EFA6F000E0D
:103B9000FB6FC4EC24F00BD00001010EF86F0A0E8D
:103BA000F96FC50EFA6F000EFB6FC4EC24F0C86B02
:103BB000C96B7CEC26F0000E046E0150045C02E13F
:103BC0000050030800010CE2800EC919006E800E3F
:103BD000005C02E1400EC85D03E2C84BC92BE9D787
:103BE0000001C86BC96B800EC919006E800E005CA5
:103BF00002E1200EC85D28E2020E046EC8C000F08B
:103C0000C9C001F00450000105E000360090013603
:103C1000FF0FF9D700011A0E0024CA6F000E012011
:103C2000CB6F7CEC26F094EC26F0CAC0E1FFCBC051
:103C3000E2FF00C0E6FF01C0E6FF02C0E6FF03C0EE
:103C4000E6FFC84BC92BCFD70001196AC86BC96BF7
:103C5000800EC919006E800E005C02E1200EC85D66
:103C60003BE2020E046EC8C000F0C9C001F004506F
:103C7000000105E0003600900136FF0FF9D7000182
:103C80001A0E0024E96E000E0120EA6EEECF00F05D
:103C9000EECF01F0EECF02F0EECF03F000C004F063
:103CA00001C005F002C006F003C007F0000E006E70
:103CB000800E016E7C0E026E880E036E4FEC23F0B8
:103CC000010ED8B0000E006E005202E0010E196E17
:103CD0000001C84BC92BBCD7120000010CB0B0EFDB
:103CE0001EF00CA258EF1FF00E6A000E0264C7EF20
:103CF0001EF0F00E0214D8A492EF1EF0023A013822
:103D00000F0B02260138F00B016E00380F0B012655
:103D10000038F00B006E08380F0B00260838F00B47
:103D2000086E0E84D89002BEABEF1EF00836003647
:103D3000013602360E2A02BEABEF1EF00836003600
:103D4000013602360E2A02BEABEF1EF008360036F0
:103D5000013602360E2A0E5003644CEF1FF0035E4C
:103D60000BBC08AE52EF1FF0D880800E0864003004
:103D7000000E002201220222D8A052EF1FF00232D0
:103D800001320032034A58EF1FF052EF1FF001C01A
:103D900002F000C001F008C000F0086A000E0E86B4
:103DA0000264FEEF1EF0F00E0214D8A4E6EF1EF03F
:103DB000023A01380F0B02260138F00B016E003871
:103DC0000F0B01260038F00B006E0E84D89002BE57
:103DD000ABEF1EF00036013602360E2A02BEABEF04
:103DE0001EF00036013602360E2A02BEABEF1EF080
:103DF0000036013602360E2AABEF1EF001C002F08B
:103E000000C001F0006A000E0E960E8802642BEFCF
:103E10001FF0F00E0214D8A416EF1FF0023A01387A
:103E20000F0B02260138F00B016E0E84D89002BEF3
:103E3000ABEF1EF0013602360E2A02BEABEF1EF0CB
:103E4000013602360E2A02BEABEF1EF001360236F4
:103E50000E2AABEF1EF001C002F0016A000E0E86C2
:103E600002645EEF1FF0F00E0214D8A43AEF1FF0C8
:103E7000023A0E84D89002BEABEF1EF002360E2A34
:103E800002BEABEF1EF002360E2A02BEABEF1EF0F2
:103E900002360E2AABEF1EF0010E0C6EEEEC26F091
:103EA00062EF1FF0020E0C6E2CEC27F062EF1FF099
:103EB000040E0C6E09EC27F062EF1FF0080E0C6E7A
:103EC00016EC27F012000001086A096A0750D8B4FE
:103ED000FAEF1FF00350D8B4FFEF1FF0025006189E
:103EE0000A6E028E068E0E6A02C008F001C00CF047
:103EF00000C00DF004500D5E0550D8A0053C0C5ECE
:103F00000650D8A0063C085E086A0C6A0D6AD8A064
:103F100091EF1FF0D8900232013200320832010EC8
:103F20000E6E0750035ED8A09EEF1FF07E0E0E248B
:103F30000326D8B004EF20F0A4EF1FF07E0E0E246D
:103F40000326D8A009EF20F0180E0B6E0D360C36A4
:103F500008360036013602360E360450005E055033
:103F6000D8A0053C015E0650D8A0063C025E06348F
:103F70000E120EA0BFEF1FF00D80CAEF1FF004500D
:103F800000260550D8B0053C01260650D8B00628BA
:103F900002260D900B2EA6EF1FF0F0EF1FF0D89029
:103FA0000036013602360E360450005E0550D8A0A9
:103FB000053C015E0650D8A0063C025E06340E1099
:103FC000010B0D26D8B00C2AD8B4082AD8A4F0EFDB
:103FD0001FF008320C320D32032AD8B404EF20F05F
:103FE0000AAE089E0850026E0C50016E0D50006E15
:103FF0000CEF20F0010E36EC27F00CEF20F0020E53
:1040000016EC27F00CEF20F0040E09EC27F00CEF73
:1040100020F0080EEEEC26F0120000010B6A0C6A8C
:104020000A6A086A0350D8B496EF20F0028E9E0EFA
:10403000035E03BE21EF20F0D8B421EF20F086EF1D
:1040400020F0036C080E035CD8A053EF20F0036E41
:10405000083600C008F001C000F002C001F0026A9A
:10406000080E035CD8A053EF20F0036E083600C0A2
:1040700008F001C000F0016A080E035CD8A053EFFD
:1040800020F0036E083600C008F0006A080E035CDA
:10409000D8A053EF20F0036E0836086A0350D8A466
:1040A000D8905FEF20F00350D8B45FEF20F0D890A5
:1040B0000232013200320832032E57EF20F00BBCDF
:1040C00008A070EF20F0D8A070EF20F0082AD8B434
:1040D000002AD8B4012AD8B4022A02BE9AEF20F0EE
:1040E0000AAE96EF20F0021E011E001E081E082ACE
:1040F000D8B4002AD8B4012AD8B4022A96EF20F006
:10410000026A016A006A086A96EF20F00B800BAE23
:10411000A0EF20F0026A0AAEA0EF20F0026E016E5E
:10412000006E086E0A360232A0EF20F0000E0C6A14
:10413000A1EF20F0010E0C6ED0EC26F0A1EF20F0E4
:10414000FF0E0250036E0150026E0050016E0850C7
:10415000006E120000010B6A0C6A086A0350D8B4A2
:104160002FEF21F002C00AF0028E9E0E035E03AE16
:104170001FEF21F0036C080E035CD8A0ECEF20F0D9
:10418000036E083600C008F001C000F002C001F064
:10419000026A080E035CD8A0ECEF20F0036E08362C
:1041A00000C008F001C000F0016A080E035CD8A04E
:1041B000ECEF20F0036E083600C008F0006A080E2D
:1041C000035CD8A0ECEF20F0036E0836086A0350B9
:1041D000D8A4D890F8EF20F00350D8B4F8EF20F02E
:1041E000D8900232013200320832032EF0EF20F074
:1041F0000BBC08A009EF21F0D8A009EF21F0082A94
:10420000D8B4002AD8B4012AD8B4022A02BE33EFA7
:1042100021F00AAE2FEF21F0021E011E001E081E23
:10422000082AD8B4002AD8B4012AD8B4022A2FEF19
:1042300021F0026A016A006A086A2FEF21F00B8000
:104240000BAE3AEF21F0026A0AAE3AEF21F0026EAD
:10425000016E006E086E0A3602323AEF21F00C6AE7
:10426000000E3BEF21F0010E0C6E000ED0EC26F09C
:104270003BEF21F0FF0E0250036E0150026E005022
:10428000016E0850006E12000CEC25F0020E0C6E50
:10429000FF0E0B6EFF0E0A6E0C2E01D007D00B2EF8
:1042A00001D003D00A2EFED7FAD7F6D7060E0B6E32
:1042B000FF0E0A6E0B2E01D003D00A2EFED7FAD7BE
:1042C0000A0E0A6E0A2EFED70E0EC16EC26A920E3A
:1042D000C06EFF0E926E936AFF0E826E020E946E97
:1042E000829E016A82BE012A000E01B0400E821831
:1042F000400B821A828E016A82BE012A000E01B032
:10430000400E8218400B821A810E0001BC6F0F0E06
:10431000BD6F6CEC22F0010E0101006F77EC24F010
:104320000C0E0101006F77EC24F0010E0001F86F14
:10433000010EF96FA9C0FAF0AAC0FBF0C4EC24F09A
:10434000020EF86F010EF96FBAC0FAF0BBC0FBF0B5
:10435000C4EC24F0100E0C6EFF0E0B6EFF0E0A6EF6
:104360000C2E01D007D00B2E01D003D00A2EFED781
:10437000FAD7F6D74C0E0B6EFF0E0A6E0B2E01D03D
:1043800003D00A2EFED7FAD7CE0E0A6E0A2EFED71B
:10439000010E0101006F77EC24F0010E0101006FA6
:1043A00077EC24F075EC1DF04EEC14F0FBD7FFD742
:1043B0000001086A096A000E076203645EEF22F0DA
:1043C000025006180A6E075003267E0ED8A0EFEFA3
:1043D00021F0035ED8B063EF22F0F3EF21F0035E2B
:1043E000D8A068EF22F0028E068E02C00EF001C047
:1043F0000BF000C00DF000500402F4CF0CF001509F
:104400000502F4CF00F0F3CF08F00402F3500C26BD
:10441000F4500822000E00220D500502F3500C2625
:10442000F4500822000E002202500402F350082625
:10443000F450002202500502016A000E0122F350DE
:104440000026F45001220D500602F3500826F450C5
:104450000022026A000E012202220B500602F350D3
:104460000026F4500122000E02220E500602F350E4
:104470000126F450022202BE46EF22F00836003632
:10448000013602360306D8B468EF22F059EF22F065
:10449000D880800E08640030000E00220122022223
:1044A000D8A059EF22F0023201320032034A63EF02
:1044B00022F00AAE029E000E6BEF22F0010E16EC07
:1044C00027F06BEF22F0020E09EC27F06BEF22F0E1
:1044D000040EEEEC26F01200BCC015F0BDC016F0C4
:1044E00015C0E1FF16C0E2FF120EE126E796E79441
:1044F000E790E79EE79CE79AE798120EE15EE79661
:10450000E794E790E79EE79CE79AE798DFEC26F0D0
:10451000E78AE788E7863BEC27F0E796DFEC26F0B2
:10452000E78AE788E7863BEC27F0E79626EC27F05A
:1045300026EC27F0E78AE788E7863BEC27F0E7964A
:10454000DFEC26F0E78AE798E7863BEC27F0E79672
:1045500026EC27F0E78AE798E7863BEC27F0E7961A
:10456000E78EE79CE7863BEC27F0E79626EC27F002
:10457000000EE76EE7863BEC27F0E796E78EE78CC8
:10458000E78AE788E7863BEC27F0E79626EC27F0FA
:10459000000EE76EE7863BEC27F0E796E788E786B4
:1045A0003BEC27F0E796DFEC26F0000EE76EE7869F
:1045B0003BEC27F0E796E78CE78AE7863BEC27F0B1
:1045C000E79626EC27F0010E176E12000C0E000184
:1045D000FE6F010EFF6F030EFE25E96E000EFF2138
:1045E000EA6EEECF00F0005001011025046E000EBF
:1045F0001121056E04C010F105C011F1800E0518DF
:10460000006E800E005C02E1000E045C05E2006AB0
:10461000016A026A036A12000101800E006E800EB8
:104620001119005C02E11051FF0827E2046A056AD3
:10463000066A076A0CC100F00DC101F00EC102F05C
:104640000FC103F04FEC23F0010ED8B0000E006E46
:10465000005209E0FF0E006EFF0E016EFF0E026EAB
:10466000FF0E036E12000001FF0E006EFF0E016EC2
:104670007F0E026EFF0E036E1200030E0001FE2578
:10468000E16E000EFF21E26E10C1E6FF0CC100F0EA
:104690000DC101F00EC102F00FC103F012000001C4
:1046A0000A6A0350D8A40A800750D8A40A820A5084
:1046B000D8B4B3EF23F0030AD8B46CEF23F00AB0F8
:1046C00067EF23F006AEB1EF23F0AFEF23F002AEB9
:1046D000AFEF23F0B1EF23F00250800B0A6E029E81
:1046E0000650800B069E0A18D8B47DEF23F00A50BE
:1046F000D8B4AFEF23F0B1EF23F00750035CD8B488
:1047000087EF23F0D8A0A3EF23F0A9EF23F0065002
:10471000025CD8B491EF23F0D8A0A3EF23F0A9EF67
:1047200023F00550015CD8B49BEF23F0D8A0A3EF91
:1047300023F0A9EF23F00450005CD8B4B3EF23F0CA
:10474000D8B0A9EF23F00A52D8B4B1EF23F0AFEFFD
:1047500023F00A52D8B4AFEF23F0B1EF23F0D880A2
:104760001200D8901200D880D884120012000001E4
:104770000D6A096A086A01500010D8B4000C015093
:1047800005180A6E0ABE0D1E0B6A05AECDEF23F0AA
:10479000041E051E042AD8B4052A01AED5EF23F065
:1047A000001E011E002AD8B4012A015005100A6E0D
:1047B0000ABEEDEF23F0C5EC25F00BB004EF24F0BA
:1047C0000DAE000C001E011E002AD8B4012A081EDE
:1047D000091E082AD8B4092A000C05AEFFEF23F001
:1047E00001BEFBEF23F00150096E0050086E016A14
:1047F000006AE0EF23F0016A006A002A000C011E43
:10480000001E0B2ADBEF23F0082AD8B4092A045033
:10481000085CD8A4E0EF23F00550095CD8A4E0EFD1
:1048200023F0096A086A002AD8B4012A01AEE0EF31
:1048300023F00000FF0C120000010D6A086A00500E
:10484000D8B4000C04180A6E0ABE0D1E0B6A04AE22
:104850002CEF24F0041E042A00A031EF24F0001EE7
:10486000002A005004100A6E0ABE58EF24F00450CB
:10487000085E003600340836045008260036060E5E
:104880000C6E00340836045000B0085E00A0082604
:1048900000360C2E41EF24F000A008260BB06AEF82
:1048A00024F00DAE000C001E002A081E082A000C81
:1048B00004AE66EF24F000BE63EF24F00050086EF3
:1048C000006A51EF24F0006A002A000C001E0B2A37
:1048D00037EF24F0082A0450085CD8A451EF24F0E4
:1048E000086A002A00AE51EF24F0FF0C120015C038
:1048F00000F016C001F000C015F001C016F015C0A0
:10490000E9FF16C0EAFF0101005300E0EF96EF94C3
:10491000EF9EEF9CEF9AEF9800BFEF8E00BDEF8CFB
:1049200000BBEF8A00B9EF881750010A02E1EF944B
:1049300002D00101EF84EF863BEC27F00101005328
:1049400000E0EF96EF94EF9EEF9CEF9AEF9800B7A0
:10495000EF8E00B5EF8C00B3EF8A00B1EF881750EF
:10496000010A02E1EF9402D00101EF840101EF8618
:104970003BEC27F0EF961750010A03E1DFEC26F03D
:1049800002D026EC27F0120010D0800E0001F86F44
:104990001AD0C00EF86F17D0940EF86F14D0D40E42
:1049A000F86F11D0800EF86F0ED00001F851010A97
:1049B000ECE0F851020AEDE0F851030AEDE0F8519D
:1049C000040AEDE0EFD7F905006EF851002600C0AB
:1049D000F8F000C000F177EC24F0176A0001FC6BDE
:1049E000FD6BFC51FA25E96EFD51FB21EA6EEECF1D
:1049F00000F000520EE0FC51FA25E96EFD51FB215A
:104A0000EA6EEECF00F177EC24F00001FC4BFD2BB9
:104A1000E8D7010E176E1200500E00019A6F6F0E4C
:104A20009B6F770E9C6F650E9D6F720E9E6F200EB2
:104A30009F6F4C0EA06F690EA16F6E0EA26F650E78
:104A4000A36F200EA46F330EA56F720EA66F640EB7
:104A5000A76FA86B9A0EA96F000EAA6F480EAB6FD6
:104A6000610EAC6F720EAD6F6D0EAE6F6F0EAF6FED
:104A70006E0EB06F690EB16F630EB26F200EB36F22
:104A80004D0EB46F650EB56F740EB66F650EB76FD1
:104A9000720EB86FB96BAB0EBA6F000EBB6F000E23
:104AA000186E000E196E120000010C6A0E6A025098
:104AB000D8A46EEF25F001C002F000C001F0006A3A
:104AC0000E860250D8A46EEF25F001C002F0016AF4
:104AD0000E960E880250D8B480EF25F00E50035E7B
:104AE000D8A4D8A086EF25F0D89002BE8CEF25F090
:104AF000003601360236032E75EF25F086EF25F0DD
:104B0000010E0C6E16EC27F090EF25F0020E0C6EE5
:104B1000EEEC26F090EF25F0040E0C6E2CEC27F056
:104B20001200000100500402F4CF09F0F3CF08F0A6
:104B300001500502F4CF0BF0F3CF0AF0005005024C
:104B4000F3500926F4500A22E86A0B2201500402AD
:104B5000F3500926F4500A22E86A0B2205AEB5EF9D
:104B600025F000500A5C01500B5801AEBCEF25F057
:104B700004500A5C05500B5808C000F009C001F051
:104B80000AC002F00BC003F0120000010134083625
:104B900009360450085E0550D8A0053C095E003671
:104BA00001360F0E0C6E013408360936045000A091
:104BB000E1EF25F0085E0550D8A0053C095EE6EF60
:104BC00025F008260550D8B0053C092600360136E8
:104BD0000C2ED3EF25F000B0F4EF25F0045008269A
:104BE0000550D8B0053C0926000012000C0E00014B
:104BF000FE6F010EFF6F030EFE25E96E000EFF2112
:104C0000EA6EEECF00F07E0E005E016A000E015AE1
:104C100010C1E1FF11C1E2FF00C0E6FF01C0E6FFE5
:104C2000030EFE25E16E000EFF21E26E7E0EE66EA3
:104C30000CC100F00DC101F00EC102F00FC103F074
:104C40001200060E0001FA6F010EFB6F01C10CF19C
:104C500002C10DF103C10EF104C10FF105C110F144
:104C6000FA0E0101116F000E126F04EC00F000C08B
:104C7000F8F001C0F9F0005001010125E16E01508A
:104C80000221E26EE66AF8C000F0F9C001F01200FD
:104C90000001FA6BFB6BFA51F825E96EFB51F92123
:104CA000EA6EEECF00F000520EE0FA51F825E96E00
:104CB000FB51F921EA6EEECFFEF01EEC27F0000169
:104CC000FA4BFB2BE8D71200000103500718D8A4B9
:104CD00079EF26F002500618D8A479EF26F001509B
:104CE0000518D8A479EF26F000500418D8B4D88459
:104CF0001200D894120012000001F86BF96B030E39
:104D0000C26E0001C2B2FDD7C4CFF8F0000EF96F39
:104D1000F8C001F0006A00C0F8F001C0F9F0C3501B
:104D20000012000E0112120000010050086E015026
:104D3000006E016A026A036A0B6A0C6A960E036EC1
:104D40000A6A00C001F008C000F0086A026A54EC68
:104D500025F0120000010050086E0150006E025054
:104D6000016E0350026E036A0B6A0C6A9E0E036E9C
:104D70000A6A020E0C6E6DEC1EF012000001086B48
:104D8000080E0C6E003408360450085ED8B0CBEF25
:104D900026F00826D89000360C2EC2EF26F012001E
:104DA00000010B800BAEDDEF26F0026A0AAEFF0EAB
:104DB000026E016E006E0A360232FF0E1200080EFD
:104DC0000B6EFF0E0A6E0B2E01D003D00A2EFED7FB
:104DD000FAD71E0E0A6E0A2EFED7120000010B84AF
:104DE0000BAEFAEF26F0010E036E026A016A006A4A
:104DF0000A360232FF0E120001010051390807E3A2
:104E0000300E005D04E3010E006E08EF27F0006A2B
:104E1000120000010B820BAE14EF27F0036802684A
:104E2000016800680A360232FF0E12000001026AB1
:104E3000016A006A086A036A000E1200176AFEC05F
:104E400000F177EC24F0010E176E1200100E0A6EBE
:104E50000A2EFED70000120000010AAE029E000ECC
:104E600012000001067E31EC17F0120000010B6AFF
:104E70000B86FF0E1200000012000000007FCDCC58
:104E80004C7B0AD723786F12037517B75171ACC5E5
:104E9000276EBD37066B95BF566777CC2B645F7066
:104EA0000961FFE65B5D08E53C3C6042221B0000B7
:104EB000007F000020820000488500007A880040C2
:104EC0001C8C0050438F002474928096189620BC4E
:104ED0003E99286B6E9CF90215A0EC782DC1CAF2A0
:104EE00049E2010000000A00000064000000E8033D
:104EF000000010270000A086010040420F008096AD
:104F0000980000E1F50500CA9A3B0100000010007E
:104F1000000000010000001000000000010000007F
:104F20001000000000010000001001000000080057
:104F3000000040000000000200000010000000809F
:104F4000000000000400000020000000000100003C
:104F500000080000004000000000303132333435DA
:104F60003637383941424344454600FF3031323309
:104F700034353637383961626364656600FF000096
:104F80000000CFBC487B5CC5477CE79F147DB6EE34
:104F9000437D785A717D99390E7E5367227EAA042B
:104FA000357EBAE3457EE9DA547E55C5617E2383BA
:104FB0006C7EDAF9747E9B147B7E5AC47E7E000080
:104FC000007F83C47E7EEC147B7E52FA747EC183A4
:104FD0006C7E18C6617ECFDB547EC0E4457ECF0573
:104FE000357E9368227EF13A0E7E515D717DB2F17D
:104FF000437DFFA2147DB3CB477CACC9487B000046
:10500000007F6EC47E7EC4147B7E16FA747E72832B
:105010006C7EB6C5617E5CDB547E3DE4457E3C051E
:10502000357EF367227E453A0E7EE55B717D34F076
:10503000437D73A1147D88C8477C3DC3487B34CF32
:105040004E6E60B6C87B31C2C77C5B9E947D38EDE6
:10505000C37D0B59F17DED388E7EB366A27E1804B8
:10506000B57E36E3C57E77DAD47EF3C4E17ED482A2
:10507000EC7E9EF9F47E7314FB7E46C4FE7E000037
:105080000000E79F147D99390E7EBAE3457E2383A5
:105090006C7E5AC47E7EEC147B7E18C6617ECF0582
:1050A000357E515D717DB3CB477CF2AFC87BB9EBE8
:1050B000C37D1366A27E04DAD47E62F9F47E00001A
:1050C000807FCAFAF47EB5DCD47ED369A27EAEF4CA
:1050D000C37D89D6C87BAFB8477CC554717D61025A
:1050E000357ECFC3617EFA137B7ED4C47E7EFE8480
:1050F0006C7ECDE6457EA13D0E7E2EA9147D00007E
:10510000007F16FA747E5CDB547EF367227E34F0F7
:10511000437D3DC3487B31C2C77C0B59F17D1804E8
:10512000B57EF3C4E17E7314FB7E97C4FE7E1184CA
:10513000EC7E43E5C57E9D3B8E7E8BA4947D671BF4
:105140009B70449B147D95370E7E30E2457E3682FF
:105150006C7E1DC47E7E65157B7E3CC7617E8507A7
:10516000357E9861717D35D5477CA69CC87B3FE72D
:10517000C37D3464A27EABD8D47EAEF8F47E46758F
:105180006E643D252E3066003372643D252E3066F8
:1051900000FF48443D252E316625252000FF0000F4
:1051A0000000A3147383FEE87184A2F933851043D1
:1051B0006D85C7211286C0392C861FA94486A63367
:1051C0005B86C3A16F868BE000877AB2088766335F
:1051D0000F87475314877A051887E3401A87000022
:1051E0001B87FB401A87AB05188790531487C6337B
:1051F0000F87F0B2088716E1008700A36F86083595
:105200005B86A2AA4486603B2C8680231286AD462C
:105210006D8561FD3385ABF07184362473830000A6
:1052200020820000208200002082000020820000F6
:1052300020820000208200002082000020820000E6
:1052400020820000208200002082000020820000D6
:1052500020820000208200002082000020820000C6
:1052600020820000208200002082000020820000B6
:1052700020820000208200002082000020820000A6
:105280001082000000820000008200000082000006
:105290000082000060810000608100006081FFFFEB
:020000040030CA
:0E000000E0FCFFFEFFFFBBFFFFFFFFFFFFFF67
:00000001FF
